:100000000C941E060C94B0270C94DD270C94460625
:100010000C94DB120C9446060C9446060C9446068F
:100020000C9446060C9446060C9446060C94460620
:100030000C9446060C9446060C9446060C94460610
:100040000C940A280C9446060C94DB2B0C941E2C62
:100050000C9446060C9446060C9446060C944606F0
:100060000C9446060C9446063B189D187C187F1885
:100070008218851888188B188E189D189718CF1914
:10008000D119D119CF19D119D119D119D119D11922
:10009000D119D119D119D119D119D119D119D11910
:1000A0005519D119D119D119D119D119C618D11988
:1000B000D119D119D119D119D119D119D119D119F0
:1000C000D119D119D119D119D119D11961196119C0
:1000D0006119611961196119611961196119D119E0
:1000E000D119D119D119D119D119C61860196019AE
:1000F00060196019D1196E1974197A198019861945
:100100008C1992199819A219AC19B619C0190719A6
:10011000C918D119D119D119D1195519D119D11914
:10012000D119D119D119D119D119D1195F195F1963
:100130005F195F19D1196E1974197A198019861906
:100140008C1992199819A219AC19B619C019071966
:10015000C918D119D119D119D1195519041A041A6C
:10016000041A041A041A041A041A041A041A041A9F
:10017000041A041A041A1B1B1B1B1B1B1B1B1B1B17
:100180001B1B491A531A5D1A671AC51ACF1ADE1AB1
:10019000EF1A771C8C1C981CA11CB01CD51CDE1CF3
:1001A000271DF01C39203F2045204C205A207C2060
:1001B0009A20456E746572206D656E752E2E2E0028
:1001C000546F67676C6564206D6963726F50504D42
:1001D00000546F67676C656420696E76657274653C
:1001E000642050504D2100546F67676C6564205443
:1001F00058206D7574696E672100546F67676C6570
:10020000642074656C656D65747279210050726F3D
:10021000746F636F6C206572726F72207769746897
:100220002052580054696D656F7574207768656E4B
:1002300020636F6E6E656374696E6720746F205201
:100240005800507265737320616E79206B65792058
:10025000746F2063616E63656C00436F6E6E6563DF
:1002600074696E6720746F2052582C20706F776508
:100270007220757020746865205258202877697440
:10028000682062696E6420706C7567206966206EF4
:100290006F74207573696E6720616C776179732064
:1002A00062696E642900546F67676C656420276912
:1002B0006D6D656469617465206F75747075742700
:1002C00000546F67676C65642027736C61766520E6
:1002D0006D6F64652700546F67676C6564202761E4
:1002E0006C776179732062696E642700546F676769
:1002F0006C65642050504D206368616E6E656C20A3
:100300006C696D69740053657420525353492069B8
:100310006E6A656374696F6E206368616E6E656C8A
:100320002028303D3D64697361626C652900536526
:10033000742050504D206D696E696D756D20737914
:100340006E630053657420626561636F6E20696E31
:1003500074657276616C0053657420626561636FC9
:100360006E2064656C617900536574206265616319
:100370006F6E206672657175656E637920696E2097
:10038000487A3A20303D64697361626C652C205074
:10039000783D504D52206368616E6E656C20782CFC
:1003A0002046783D465253206368616E6E656C202E
:1003B00078005365742050574D2073746F7020641B
:1003C000656C61792028302064697361626C6564B2
:1003D0002C20312D323535203D3D20302E317320FB
:1003E0002D2035306D696E29005365742050504DB5
:1003F0002073746F702064656C61792028302064EC
:10040000697361626C65642C20312D323535203D75
:100410003D20302E3173202D2035306D696E29003E
:10042000536574206661696C736166652064656CF0
:1004300061792028302064697361626C65642C20C6
:10044000312D323535203D3D20302E3173202D2089
:1004500035306D696E29002A2A2A2A2A2A2A2A2A50
:100460002A2A2A2A2A2A2A2A2A2A2A2A2A2A2A2AEC
:100470002A2A2A2A0052582041636B6564202D20C5
:1004800072657665727420737563636573736675E0
:100490006C21002A2A2A2A2A2A2A2A2A2A2A2A2AAD
:1004A0002A2A2A2A2A2A2A2A2A2A2A2A2A2A2A2AAC
:1004B000002A2A2A2A2A2A2A2A2A2A2A2A2A2A2AC6
:1004C0002A2A2A2A2A2A2A2A2A2A2A2A2A2A00528E
:1004D000582041636B6564202D20757064617465DC
:1004E000207375636365737366756C21002A2A2A0D
:1004F0002A2A2A2A2A2A2A2A2A2A2A2A2A2A2A2A5C
:100500002A2A2A2A2A2A2A2A2A2A0056616C696457
:100510002063686F69636573206172653A205B319F
:100520005D2D5B31365D20286368616E6E656C20E1
:10053000312D31362900536574206F7574707574D0
:1005400020666F7220706F727420005B585D2061AE
:10055000626F7274206368616E67657320616E6498
:10056000206578697420525820636F6E6669670051
:100570005B535D20736176652073657474696E6783
:100580007320746F205258005B525D20726576654F
:1005900072742052582073657474696E6773207486
:1005A0006F2064656661756C747300557365206EA9
:1005B000756D62657273205B312D445D20746F2010
:1005C0006564697420706F727473205B452D515D92
:1005D00020666F722073657474696E677300202DD6
:1005E00020726563656976657220636F6E66696700
:1005F000757261746F722C20727820737720000AF4
:100600000A6F70656E4C52536E67200053657420FC
:1006100073657269616C2062617564726174653AB8
:10062000200056616C69642063686F696365733A82
:100630002031202D20342B34202F2032202D203823
:10064000202F2033202D20382B34202F2034202D14
:10065000203132202F2035202D2031322B34202FF5
:100660002036202D20313600536574204368616E9A
:100670006E656C20636F6E6669673A20005365741F
:100680002044617461726174652028302D32293AEA
:10069000200053657420486F70206368616E6E653A
:1006A0006C7320286D61782032342C207365706162
:1006B000726174656420627920636F6D6D61732966
:1006C0002076616C69642076616C75657320312DCC
:1006D0003235353A2000536574206368616E6E656B
:1006E0006C2073706163696E6720287831306B48C5
:1006F0007A293A200053657420524620706F77653E
:10070000722028302D37293A200053657420524634
:10071000206D6167696320286865782920652E67E8
:100720002E20307844454144463030443A2000532E
:1007300065742062617365206672657175656E63AC
:10074000792028696E20487A293A20005B5A5D207A
:10075000656E746572207265636569766572206383
:100760006F6E66696775726174696F6E2075746902
:100770006C79005B465D20646973706C61792061FF
:10078000637475616C206672657175656E63696509
:10079000732075736564005B525D2063616C6375E3
:1007A0006C6174652072616E646F6D206B65792079
:1007B000616E6420686F70206C697374005B495DC2
:1007C000207265696E697469616C697A6520736508
:1007D0007474696E677320746F20736B65746368DB
:1007E0002064656661756C7473005B585D2072658A
:1007F00076657274206368616E67657320616E64EC
:100800002065786974206D656E75005B535D20739B
:100810006176652073657474696E677320746F20E8
:10082000454550524F4D20616E64206578697420B3
:100830006D656E7500557365206E756D62657273BA
:10084000205B302D395D20746F20656469742070E1
:100850006172616D657465727300202D2053797328
:1008600074656D20636F6E66696775726174696F18
:100870006E000A0A6F70656E4C52536E672000510D
:1008800029204F7574707574206265666F726520DB
:100890006C696E6B20283D465329203A2000502970
:1008A00020536C617665206D6F64652028657870D3
:1008B0006572696D656E74616C293A20004F29205C
:1008C00054696D65642042494E44206174207374FC
:1008D000617274757020203A20004E292050504DCE
:1008E000206F7574707574206C696D69746564200F
:1008F000202020203A200044495341424C454400E6
:100900004D292050504D205253534920746F20637D
:1009100068616E6E656C202020203A20004C2920F2
:1009200050504D206D696E696D756D2073796E63E1
:10093000202875732920203A200044495341424C15
:100940004544004B29204661696C736166652062ED
:100950006561636F6E20696E74762E2028312D32AA
:10096000353573293A20004A29204661696C736144
:10097000666520626561636F6E2064656C617920D5
:1009800028302D323535203D3E20313073202D204A
:100990003135306D696E293A200049292046616958
:1009A0006C7361666520626561636F6E206672714B
:1009B0002E203A200048292050574D2073746F7024
:1009C0002064656C6179202020202020203A2000BE
:1009D00047292050504D2073746F702064656C61FE
:1009E00079202020202020203A200046292046611E
:1009F000696C736166652064656C617920202020D4
:100A00002020203A200050574D206368616E6E65AB
:100A10006C200066756E6374696F6E3A2000292041
:100A2000706F72742000506F776572546F776572C3
:100A300000445446205548462033322D62697420C4
:100A400031306368004F70656E4C52536E67525878
:100A5000206D696E6920342F36636800466C7974A6
:100A6000726F6E2F4F72616E6765525820554846FF
:100A70002038636800525820747970653A20004429
:100A8000697361626C656400487A00203D3D200016
:100A900043616C63756C61746564207061636B6540
:100AA0007420696E74657276616C3A200042292068
:100AB0004D6963726F202868616C66292050504D23
:100AC000202020203A00412920496E766572746505
:100AD000642050504D20696E20202020203A0030A4
:100AE00029204D7574652062757A7A657220286DAB
:100AF0006F73746C79293A003929205365726961E2
:100B00006C2062617564726174653A00736D617224
:100B100074506F7274004672536B79005472616E38
:100B200073706172656E740044697361626C6564B0
:100B30000038292054656C656D657472793A2020FF
:100B40002020202020003729204368616E6E656CCC
:100B500020636F6E6669673A202000362920446161
:100B60007461726174652028302D32293A2020206A
:100B700000352920486F70206368616E6E656C7364
:100B80003A2020202020003429204368616E6E65C1
:100B90006C2073706163696E673A202000332920EE
:100BA000524620706F7765722028302D37293A2001
:100BB0002020003229205246206D616769633A2067
:100BC0002020202020202020003129204261736530
:100BD000206672657175656E63793A202020000089
:100BE00000000700020100000304060000000000EE
:100BF00000000001020408102040800102040810D7
:100C00002001020408102004040404040404040263
:100C10000202020202030303030303000000002395
:100C2000002600290000000000250028002B0000FD
:100C3000000000240027002A00000C2D11241FBEF4
:100C4000CFEFD8E0DEBFCDBF13E0A0E0B1E0E6E239
:100C5000F0E602C005900D92A83CB107D9F716E066
:100C6000A8ECB3E001C01D92AC38B107E1F71CE07D
:100C7000CCE3DCE004C02297FE010E94152ECA33AB
:100C8000D107C9F70E94482D0C9411300C94000034
:100C900080917105813019F482E080937105809113
:100CA0007105833019F484E0809371050895A89547
:100CB0000895DC01ED91FC910190F081E02D099502
:100CC00008952091720530917305382748E0C901D5
:100CD000880F991F37FF06C09C0151E2252750E17C
:100CE000352701C09C01415091F730937305209343
:100CF0007205089588E38093740580E092ECA1E08A
:100D0000B0E08093750590937605A0937705B09336
:100D1000780587E08093810580EC92E9ADEEB9E13A
:100D20008093790590937A05A0937B05B0937C0519
:100D300085E0809382058DEE9EEFADEABEED809357
:100D40007D0590937E05A0937F05B0938005E3E831
:100D5000F5E080E090E0863028F4DC01AF54BC4F31
:100D60002C9101C020E0219301968831910599F7DB
:100D700082E080939B058AE080939C05089580EC37
:100D800091EDA8E9BBE18093B9059093BA05A093D2
:100D9000BB05B093BC0580E090E0A0E0B0E5809397
:100DA000BD059093BE05A093BF05B093C005E1ECCF
:100DB000F5E080E081938F5F8031E1F70895A0E056
:100DC000B0E0E5EEF6E00C94DE2DD82F0E9460280E
:100DD0006115710581059105C9F30E94812E10925C
:100DE0007D0510927E0510927F0510928005C4E06B
:100DF000812C912C54018A94C0907D05D0907E0561
:100E0000E0907F05F0908005FE2CED2CDC2CCC24AE
:100E10000E947C2EA50194010E94BD2D6C0D7D1DAC
:100E20008E1D9F1D60937D0570937E0580937F05C9
:100E300090938005C15001F7DD2309F450C003E809
:100E400015E0E801A12CB12C62E3C62ED12CE12CD7
:100E5000F12C8881882309F442C0B39419F40E94CC
:100E60007A063DC00E947C2EA70196010E94BD2DEE
:100E7000E1E0E60FA3E8B5E08A2F801B8A1520F495
:100E80008D918E13F9CFE9CF2091820530E0A0E15A
:100E9000B7E20E94552D9B01AC01AE2FB0E00E943D
:100EA000642D4090790550907A0560907B05709094
:100EB0007C05640D751D861D971D4090B9055090E9
:100EC000BA056090BB057090BC05461657066806CB
:100ED000790618F2E993A39488E1A812BACFCDB7A6
:100EE000DEB7E0E10C94FA2D8436910520F4BC01C4
:100EF00080E090E017C09C018E3B910528F42A55B4
:100F00003109AAE0B0E00CC0823D910528F4245BD1
:100F10003109A4E6B0E004C02D5C3109A8E5B2E0D7
:100F20000E94552DA4E6B0E09B01AC010E94642D07
:100F3000089590E08C599F4F0E947407089561E0D6
:100F400089E00E940D2960E089E00E944629089509
:100F5000892B11F061E001C060E089E00E94462920
:100F6000089560E08EE00E940D2961E08FE00E940C
:100F70000D2961E082E00E940D2960E083E00E947B
:100F80000D2961E084E00E940D29089542E050E0BF
:100F900068E476E081E00E9490270895E3E0F0E0C5
:100FA00089E080935700E491E67081E0E63009F033
:100FB00080E00895CF93DF93C82F0E94CE07882347
:100FC00081F0DFB781E080937005F8940E945706A6
:100FD00088E180936000C0936000C1110E945706B1
:100FE000DFBFDF91CF9108958F929F92AF92BF9212
:100FF000CF92DF92EF92FF92CF93FC01C0A5EC2F2E
:10100000E770F0E0E758FC4FA081B0E0C7FF03C0F5
:1010100024E130E002C02FE030E0FC0197A183E141
:10102000989FF0011124E25CFE4F80809180A280A5
:10103000B380A20FB31F20E43FE14DE750E00E94D0
:101040006F2DA50194010E949B2D8C2F887149F46E
:1010500069017A01E0EDCE0EE7E0DE1EE11CF11C35
:101060001BC0C7FF05C060E47AE88CE29EE004C0C4
:1010700060E07EEE8AEB9BE069017A01F8EBCF0E2F
:10108000FBE0DF1EE11CF11CA50194010E949B2DD9
:10109000C20ED31EE41EF51EC701B60169517C4F76
:1010A0008F4F9F4F28EE33E040E050E00E949B2D91
:1010B000A8EEB3E00E94642DCF91FF90EF90DF90F7
:1010C000CF90BF90AF909F908F9008958F3F9105E4
:1010D00051F048F0811522E0920738F081159340D5
:1010E00030F482E0089580E0089581E0089583E07F
:1010F0000895A0E0B0E0EFE7F8E00C94E72DEB01F5
:101100008A01B82FB695A0E028813981F8012083A3
:101110002A813B8121832C813D8122832E813F8145
:101120002383688179814A815B812C813D81EE81B5
:10113000FF819F2F9295990F990F907C272F2370F5
:10114000922B252F2370220F220F922B232F2370F7
:101150002295207F922BF80194830B5F1F4F2896D6
:10116000AF5FBA1788F680FF24C0888199810E94FA
:101170006608D82E8A819B810E946608E82E8C81A1
:101180009D810E946608F82E8E819F810E946608CC
:10119000F0E4DF9EA001112490E1E99E900111246A
:1011A000242B282BE4E0FE9EB0011124262BF8010D
:1011B0002083CDB7DEB7E7E00C94032E803223E026
:1011C000920708F1883E23E0920740F48F51934044
:1011D000E4E096958795EA95E1F70895803D27E04C
:1011E000920718F48C5D93400895883928E092079F
:1011F00068F4885C974074E0969587957A95E1F756
:101200008D509C4F089580E090E008958FEF93E01B
:1012100008958C30910540F4A4E0880F991FAA9599
:10122000E1F7885D9C4F0895843F23E0920718F40E
:1012300084529C4F0895811524E0920740F486570C
:10124000934FF4E0880F991FFA95E1F7089580E92C
:1012500098E008959C013695279525753575821B74
:10126000930B9C0123733373969587959695879579
:1012700083739373820F931F9C0154E036952795D7
:101280005A95E1F7280F391F2F703F7041E051E068
:10129000249FC001259F900D349F900D1124892F0C
:1012A00008955A98882319F00000419A02C000005E
:1012B000419800005A9A000008955A9A000086B199
:1012C0005A98000081700895CF93DF93D82F5C9ACD
:1012D0005A985C98C8E08D2F80780E945109DD0FE4
:1012E000C150C9F75A98DF91CF9108958F770E9426
:1012F00064090895CF93DF93D82FC8E08D2F8078AD
:101300000E945109DD0FC150C9F75A98DF91CF9162
:101310000895CF93DF935A98C8E080E0D82FDD0F6F
:101320000E945D098D0FC150C9F7DF91CF910895DB
:101330000E9476090E9489095C9A0895A1E0B0E0B4
:10134000E4EAF9E00C94EC2D806869830E9464095A
:101350006981862F0E947A095C9A2196E2E00C94BA
:10136000082ECF93C0917D05C827E82FF0E0EC58F8
:10137000FA4F678589E70E949E096C2F8DE30E94D2
:101380009E096C2F82E40E949E09CF91089586E207
:101390000E9498090895CF93DF93EC016C818CE152
:1013A0000E949E096D818DE10E949E096E818EE1F1
:1013B0000E949E096F8180E20E949E09688581E2F9
:1013C0000E949E09698582E20E949E096A8583E2E5
:1013D0000E949E096B8584E20E949E096C8585E2CD
:1013E0000E949E096D858AE20E949E096E858EE6A6
:1013F0000E949E096F858FE60E949E09688980E79A
:101400000E949E09698981E70E949E096A8982E794
:101410000E949E09DF91CF910895CF92DF92EF92C3
:10142000FF92CF93DF936B017C01C11488E3D80650
:101430008CE9E8068CE1F80628F5C701B60120E83A
:1014400036E948E950E00E949B2DE901689760E881
:1014500079E687E69FEF0E94772D6C0D7D1D8E1D2E
:101460009F1DF2E0660F771F881F991FFA95D1F72D
:1014700021E732E040E050E00E949B2DF22EE32E67
:1014800080E421C0C701B60120E03DE241E351E024
:101490000E949B2DE901689760E073ED8EEC9EEF52
:1014A0000E94772D6C0D7D1D8E1D9F1D660F771F71
:1014B000881F991F21E732E040E050E00E949B2DF9
:1014C000F22EE32E80E66C2F6F71680F85E70E9485
:1014D0009E096E2D86E70E949E096F2D87E70E9468
:1014E0009E09DF91CF91FF90EF90DF90CF9008950C
:1014F000682F8DE60E949E0908958F929F92AF9269
:10150000BF92CF92DF92EF92FF92CF93DF93D82FCB
:1015100083E00E94980980936F0584E00E949809F7
:1015200080936E0560E086E00E949E0961E087E09E
:101530000E949E096FE789E00E949E0965E08AE0AB
:101540000E949E0962E18BE00E949E0965E18CE0A9
:101550000E949E096DEF8DE00E949E0960E08EE082
:101560000E949E09DD2319F08BE291E008C02091D2
:101570009B0533E1239FC0011124825C9E4F0E9492
:10158000CB096CE880E30E949E096FE082E30E9431
:101590009E0962E483E30E949E0980919C0587FF77
:1015A00002C064E101C06AE084E30E949E096AE22D
:1015B00085E30E949E096DE286E30E949E0964ED28
:1015C00087E30E949E0960E088E30E949E0960E034
:1015D00089E30E949E09D11109C0C0907D05D09079
:1015E0007E05E0907F05F090800507C0C5E9CC2E10
:1015F000C1ECDC2EED2CCEEDFC2ECAE38F2C992411
:10160000AA24BB24682D8C2F0E949E09682D85E09A
:101610008C0F0E949E09FE2CED2CDC2CCC24CF5F7D
:10162000CE3361F76FEF83E40E949E096FEF84E48D
:101630000E949E096FEF85E40E949E096FEF86E489
:101640000E949E09DD2311F066E002C060918105D1
:101650008DE60E949E0960E089E70E949E096091E4
:1016600082058AE70E949E0960E083E70E949E0946
:1016700060E084E70E949E09D11109C0609179055C
:1016800070917A0580917B0590917C0504C060EC97
:1016900072E98DEE99E10E940D0ADF91CF91FF90E2
:1016A000EF90DF90CF90BF90AF909F908F90089574
:1016B00061E087E00E949E0964E28EE70E949E0935
:1016C00063E088E00E949E0960E088E00E949E0935
:1016D00065E087E00E949E0962E085E00E949E0925
:1016E00083E00E94980980936F0584E00E94980926
:1016F00080936E05089583E00E94980980936F059A
:1017000084E00E94980980936E0561E087E00E9462
:101710009E096AE070E080E090E00E9483280E94C9
:10172000580B00000895CF92DF92FF920F931F9302
:10173000CF93DF931F92CDB7DEB7082F162F8EE31E
:1017400099830E949E09F02EC02E9981D92E8C2D4E
:101750008F19811738F4F60161916F018FE70E94AC
:101760009E09F5CF64E085E00E949E0983E00E9417
:10177000980980936F0584E00E94980980936E0514
:101780000E94602860936A0570936B0580936C05D6
:1017900090936D0569E087E00E949E0981E0809347
:1017A00071050F90DF91CF911F910F91FF90DF9006
:1017B000CF9008950F931F930E94930B8091710512
:1017C000813099F40E94602800916A0510916B05A0
:1017D00020916C0530916D05601B710B820B930B92
:1017E000603A76488140910548F3809171058130D7
:1017F00031F46DE971E080EE95E00E942F2A1F918F
:101800000F9108950F931F9380917105823021F4F9
:101810001092710581E020C0809171058130D9F46A
:101820000E94602800916A0510916B0520916C055B
:1018300030916D05601B710B820B930B613A7648FA
:101840008140910540F061E087E00E949E0910927E
:10185000710582E001C080E01F910F910895CF9340
:10186000DF93EC014AE050E06D2F70E080EE95E0F0
:101870000E94FD2A6EE280EE95E00E94012ABE01E0
:1018800084E0769567958A95E1F76F7077274AE04F
:1018900050E080EE95E00E94FD2ADF91CF910895FF
:1018A000D82FC0E0CD1780F42C9A64E670E080E079
:1018B00090E00E9483282C9864E670E080E090E03D
:1018C0000E948328CF5FEECF6CE271E080E090E071
:1018D0000E948328E6CF0F931F93CF93DF93EC01F1
:1018E000062F15E0115051F0CE010E94F82F081775
:1018F00041F0602FCE010E940030F4CF82E00E94C0
:10190000500CDF91CF911F910F910895A0E0B0E0AE
:10191000ECE8FCE00C94DE2D482E562EC0E0D0E022
:10192000612C712CE12CF12C00E010E041100CC076
:101930006090D20586E4689E3001112459E1E52EBD
:10194000F12C08EB15E01EC091E049120FC0609029
:10195000D205E6E46E9E30011124FBE16F0E711C8E
:1019600049E2E42EF12C04E715E00CC082E04812B5
:1019700009C028E1622E77247394EE24E394F12CBD
:1019800001ED15E043018C0E9D1E1092730510921F
:1019900072053401A62CA818B12CC30101966C0164
:1019A000AE14BF04A8F4A00EB11E511006C0C301AE
:1019B0000E94F82FF501808305C0F5016081C30105
:1019C0000E946B0CF50180810E9461063601E2CF16
:1019D000C301511018C0C3010E94F82FB82EC601D0
:1019E0000E94F82F2B2D30E0322F2227282B8091B8
:1019F0007205909173058217930779F4C0E0D0E0E7
:101A00005524539493CF3601609173050E946B0C5B
:101A100060917205C6010E946B0CC05EDE4FC13E34
:101A200092E0D90708F482CF852DCDB7DEB7E0E18B
:101A30000C94FA2D61E082E00E94860C089560E02B
:101A400082E00E94860C8091D105853028F084E0E8
:101A50008093D1050E941A0D8091D1058093D20503
:101A6000089561E080E00E94860C61E081E00E94C0
:101A7000860C089560E080E00E94860C882351F077
:101A800060E081E00E94860C882321F0809174053B
:101A9000883349F00E94BF060E947A0681E00E94C6
:101AA000DF060E94310D0895882319F069EA71E07C
:101AB00002C06DEA71E080EE95E00E942F2A089541
:101AC000FF920F931F93CF93DF9369EC7BE080EE3F
:101AD00095E00E94DB294091790550917A0560914B
:101AE0007B0570917C052AE030E080EE95E00E9455
:101AF000042B63EB7BE080EE95E00E94DB294091B4
:101B00007D0550917E0560917F057091800520E1F3
:101B100030E080EE95E00E94042B6DE97BE080EEE2
:101B200095E00E94DB294AE050E06091810580EE5B
:101B300095E00E942C2B67E87BE080EE95E00E9408
:101B4000DB294AE050E06091820580EE95E00E943A
:101B50002C2B61E77BE080EE95E00E94DB29C3E857
:101B6000D5E0F12C8E0188818823A9F0FF2031F087
:101B700060EB71E080EE95E00E94FE2921964AE03C
:101B800050E0F801608180EE95E00E94F52AF39420
:101B9000F8E1FF12E7CF80EE95E00E94092A6BE59D
:101BA0007BE080EE95E00E94DB294AE050E0609106
:101BB0009B0580EE95E00E942C2B66E47BE080EE96
:101BC00095E00E94DB29E0919C05E770F0E0EE0FC4
:101BD000FF1FEF57FC4F6081718180EE95E00E94FE
:101BE0002F2A61E37BE080EE95E00E94DB29809163
:101BF0009C058871883069F028F4811113C068E26F
:101C00007BE00CC0803141F0883161F46CE07BE016
:101C100005C06CE17BE002C066E17BE080EE95E010
:101C20000E941D2A68EF7AE080EE95E00E94DB2991
:101C30004091750550917605609177057091780512
:101C40002AE030E080EE95E00E94042B6FED7AE010
:101C500080EE95E00E94DB298091BD0580710E9495
:101C6000540D66EC7AE080EE95E00E94DB298091CD
:101C7000BD0580740E94540D6DEA7AE080EE95E017
:101C80000E94DB298091BD0580720E94540D60E99D
:101C90007AE080EE95E00E94DB2984E795E00E94DF
:101CA000F407AB01BC012AE030E080EE95E00E9431
:101CB000E62A6BE87AE080EE95E00E94DB2984E773
:101CC00095E00E94F4079B01AC0160E472E48FE0B0
:101CD00090E00E949B2DBA01A9012AE030E080EE3D
:101CE00095E00E94E62A68E87AE080EE95E00E949E
:101CF0001D2ACDB7DEB7E5E00C94052E8F929F929A
:101D0000AF92BF92CF92DF92EF92FF92811107C004
:101D10006FE77AE080EE95E00E941D2A2FC090E0E8
:101D20000E94740724E630E040E050E00E949B2DC2
:101D3000CA01B9012AE030E040E050E00E949B2D4A
:101D400049015A016B017C012AE030E0B501A40190
:101D500080EE95E00E94E62A6EE280EE95E00E9419
:101D6000012A2AE030E0B701A60180EE95E00E944A
:101D7000E62A63E780EE95E00E94412AFF90EF900B
:101D8000DF90CF90BF90AF909F908F9008951F935A
:101D9000CF93DF9365E77AE080EE95E00E94DB2940
:101DA00080919D05813041F46CE57AE080EE95E00C
:101DB0000E941D2A10E050C0823019F465E47AE0D8
:101DC000F5CF843019F461E37AE0F0CF853091F7F4
:101DD00066E27AE0EBCFC12FD0E0C930D1050CF438
:101DE00041C068E3610F80EE95E00E94012A6EE138
:101DF0007AE080EE95E00E94DB29BE016F5F7F4FA5
:101E00004AE050E080EE95E00E94C52A63E17AE066
:101E100080EE95E00E94DB29C356DA4FE981E0327B
:101E200018F566E07AE080EE95E00E94DB29898172
:101E3000803130F06CE673E080EE95E00E94FE2980
:101E400069816F7070E06F5F7F4F4AE050E080EE15
:101E500095E00E94CE2A1F5F80914605181708F46E
:101E6000BACF0FC061E3BECFEF70F0E0EE0FFF1FFF
:101E7000EF56FC4F6081718180EE95E00E942F2A21
:101E8000EACF6BEE79E080EE95E00E94DB2980914D
:101E9000B5050E947E0E60ED79E080EE95E00E942F
:101EA000DB298091B6050E947E0E65EB79E080EE1D
:101EB00095E00E94DB298091B7050E947E0E6AE9B9
:101EC00079E080EE95E00E94DB294091AD055091CC
:101ED000AE056091AF057091B005411551056105E2
:101EE000710539F12AE030E080EE95E00E94042B84
:101EF00067E679E080EE95E00E94DB298091B105EC
:101F00000E949907AB01BC012AE030E080EE95E029
:101F10000E94042B63E479E080EE95E00E94DB29C7
:101F20004AE050E06091B20580EE95E00E942C2BD3
:101F300006C06AE379E080EE95E00E941D2A6DE11B
:101F400079E080EE95E00E94DB296091B305709105
:101F5000B4054AE050E080EE95E00E94162B60E068
:101F600079E080EE95E00E94DB296091AC05603459
:101F700050F470E06F5F7F4F4AE050E080EE95E0F4
:101F80000E94CE2A06C067EF78E080EE95E00E94BE
:101F90001D2A6AED78E080EE95E00E94DB298091B1
:101FA000AB0580FF03C062EB71E002C066EB71E03D
:101FB00080EE95E00E942F2A6DEB78E080EE95E0B0
:101FC0000E94DB298091AB0582700E94540D6EE95E
:101FD00078E080EE95E00E94DB298091AB0584706B
:101FE0000E94540D6FE778E080EE95E00E94DB29B7
:101FF0008091AB0588700E94540DDF91CF911F91A5
:1020000008950F931F93CF93DF93209143052F3FA4
:10201000A9F56FEF75E080EE95E00E94DB2980E87E
:1020200093E00E942F0C6EED75E080EE95E00E942B
:10203000DB2980914405909145050E942F0C6BEAA5
:1020400075E080EE95E00E941D2A68E875E080EE5C
:1020500095E00E941D2A60E775E080EE95E00E9401
:102060001D2A6BE475E080EE95E00E941D2A80EE4B
:1020700095E00E94092A0E94C70E68C012160CF053
:1020800065C0332727FD30958091460590E0821783
:1020900093070CF45BC066E375E080EE95E00E9468
:1020A000DB2960914305772767FD70954AE050E092
:1020B00080EE95E00E94CE2A6BE075E080EE95E020
:1020C0000E94DB2910E008E2809147051817D0F53F
:1020D000C12FD0E0CC0FDD1FC85BDA4F288130E084
:1020E00080914305992787FD909501972817390717
:1020F00039F56AEB71E080EE95E00E94FE294AE036
:1021000050E0602F80EE95E00E94F52A6EEB71E0C2
:1021100080EE95E00E94FE29E981EF70F0E0EE0F7D
:10212000FF1FEF56FC4F6081718180EE95E00E94A9
:10213000FE2962EC71E080EE95E00E94FE290F5FBF
:102140001F5FC2CF80EE95E00E94092ADF91CF91F8
:102150001F910F910895FF920F931F93CF93DF93D9
:10216000C3E8D5E0F12C8E0188818823D1F164EC9D
:1021700071E080EE95E00E94FE294AE050E06F2D6C
:1021800080EE95E00E94F52A61ED71E080EE95E029
:102190000E94FE292196F801208130E0A0E1B7E2FB
:1021A0000E94552D9B01AC01A0918205B0E00E94D8
:1021B000642DAB01BC018091790590917A05A091C5
:1021C0007B05B0917C05480F591F6A1F7B1F2AE0D1
:1021D00030E080EE95E00E94042BF394F8E1FF12CA
:1021E000C2CFCDB7DEB7E5E00C94052E1092DD042A
:1021F00085E6EEEDF4E0DF011D928A95E9F708959A
:10220000CF93C82F8F3719F0883009F045C0E0917F
:10221000DD04EE23D9F1E150E093DD04F0E0E25279
:10222000FB4F10826DE070E080EE95E00E94590651
:10223000C0E08091DD04C81760F4EC2FF0E0E252BA
:10224000FB4F608170E080EE95E00E945906CF5F01
:10225000F0CF60E270E080EE95E00E9459066DE0FC
:1022600070E080EE95E00E945906C0E08091DD04A8
:10227000C81778F5EC2FF0E0E252FB4F608170E078
:1022800080EE95E00E945906CF5FF0CF67E080EEC8
:1022900095E00E94012A1DC08B3119F40E94F610AE
:1022A0001AC08D30C1F08A30B1F08091DD048436DF
:1022B00068F76C2F70E080EE95E00E945906E0917F
:1022C000DD0481E08E0F8093DD04F0E0E252FB4FED
:1022D000C08380E001C081E0CF910895CF93C82FE3
:1022E0000E9460286093C6047093C7048093C8045A
:1022F0009093C904C093DB04CC2329F040E051EE55
:1023000060E070E004C040E855E260E070E080EE1C
:1023100095E00E948B2CCF9108959091CA04492F8B
:102320004F7050E0BA016F5F7F4F292F30E0E4E03B
:1023300035952795EA95E1F76217730759F0FA0189
:10234000E553FB4F808381E0890F8F70907F892B4D
:102350008093CA0408956EE770E080EE95E00E94D5
:1023600059060895A3E1B1E0E8EBF1E10C94DF2D0B
:10237000E3E8F5E0712C8191882321F0739428E142
:102380007212F9CF65ED71E080EE95E00E942F2A80
:102390004AE050E0672D80EE95E00E942C2B80E013
:1023A0000E947D0A0E94580B8E010E5F1F4FC12CA8
:1023B000D12C7601C39466246A945C2C0E94542824
:1023C0004B015C012091820530E0A0E1B7E20E9460
:1023D000552D9B01AC01C701B6010E94772D2091BC
:1023E000790530917A0540917B0550917C05620F0B
:1023F000731F841F951F2091B9053091BA05409134
:10240000BB055091BC05261737074807590718F434
:10241000F801608225C08C2D0E94B10961E070E056
:1024200080E090E00E948328F80110820E945428E6
:10243000681979098A099B09643F714081059105F2
:1024400040F40E94C709F8019081981778F78083BB
:10245000EDCF50FE03C02B982C9A02C02B9A2C98DB
:102460002FEFC21AD20AE20AF20A0F5F1F4F8FEF54
:10247000C816D104E104F10409F09FCFCE01939571
:10248000FC01D82E7FEF68EC2E2F281B271510F0AB
:1024900051E056C0DE01129651E02FEF41E03D9130
:1024A000321710F0322F01C0452F5F5F5F3F11F0F0
:1024B000232FF5CF4193242F30E0A1E0B0E0AC0F03
:1024C000BD1FA20FB31F5C93413079F0DE01A20F54
:1024D000B31F5C93423049F0AFEFBFEFAC0FBD1FAD
:1024E000A20FB31F6C934E3F78F6A2E0B0E0AC0FA2
:1024F000BD1FA20FB31F7C934D3F30F6A3E0B0E0A9
:10250000AC0FBD1FA20FB31F6C93BECF452F242F5E
:1025100030E0FC01E20FF31F6081AFEFB0E0AC0FE1
:10252000BD1FA20FB31F2C91621748F44150DC016C
:10253000A40FB11D2C9120836C934111E8CF5F5FF4
:10254000571520F3372D369520E0231770F4DC0162
:10255000A20FB11D4C91522F530FFC01E50FF11D3D
:1025600050815C9340832E5FF0CFF3E8EF2EF5E0CF
:10257000FF2E8C01802F8D19871598F4F801C190DA
:102580008F014AE050E06C2D80EE95E00E94F52A24
:102590006CE280EE95E00E94012AF701C1927F0172
:1025A000E9CF80EE95E00E94092A81E0CD5EDE4F02
:1025B000EFE00C94FB2D1F920F920FB60F92112497
:1025C0000F931F932F933F934F935F936F937F933B
:1025D0008F939F93AF93BF93EF93FF934091BD056C
:1025E0005091BE056091BF057091C00586B18A010A
:1025F0009B01007411272227332785FB882780F948
:1026000090E0A0E0B0E0081719072A073B0709F49B
:1026100068C080918400909185001092850010928E
:1026200084002091A70421115CC045FD02C096954D
:102630008795853C29E09207C0F180910A0190E0DE
:10264000A0E0B0E00CE176956795579547950A951F
:10265000D1F7411551056105710521F441E050E0C4
:1026600060E070E0481759076A077B07D8F480914B
:102670000A018F3FB9F040E080910A01481780F4C9
:10268000842F90E0880F991FFC01E957FB4F2081B0
:102690003181FC01E55FFE4F318320834F5FECCF3A
:1026A0001092A80410920A011CC08D3B22E09207F0
:1026B000A8F020910A01203188F410910A0121E04C
:1026C000210F20930A010E94DE08E12FF0E0EE0FB7
:1026D000FF1FE957FB4F9183808303C08FEF8093E7
:1026E0000A01FF91EF91BF91AF919F918F917F91DF
:1026F0006F915F914F913F912F911F910F910F908B
:102700000FBE0F901F90189583E0809380008AE1A0
:10271000809381008FEF9FEF9093890080938800D2
:1027200010926F0080E280936C00E8E6F0E0808118
:102730008260808308950E941F0D8091D2058430AD
:1027400011F41092D20508956F3018F086958058D4
:10275000089589E0689F802D11240895A0E0B0E0DD
:10276000E4EBF3E10C94E62DC82F0E946028009161
:1027700038041091390420913A0430913B046B01E4
:102780007C01C01AD10AE20AF30A9701860149E8DE
:10279000C41643E1D406E104F10410F010923C04A5
:1027A000609338047093390480933A0490933B0407
:1027B0002091A7048FEF820F8230D8F5E0913C047E
:1027C000EE2309F44EC1E13011F482E0B8C1E031EA
:1027D00008F034C181E08E0F80933C04F0E0E957AB
:1027E000FB4FC083803109F0ACC1E9E8F4E021304F
:1027F00029F4A181A695A695808108C08081918148
:10280000A92FA695A695A69596958795A03148F4EB
:10281000B0E090E0AA0FBB1FA55FBE4F11969C933E
:102820008E931092A804329684E0E739F807F9F6FF
:1028300088C1233009F005C1E0913C04E11104C0D6
:10284000CF3009F07EC10DC1E83148F481E08E0F30
:1028500080933C04F0E0EA57FB4FC08372C1E8313B
:1028600009F0ECC0C111EAC040E050E0ABE0CA01A1
:10287000B3E0880F991FBA95E1F7A49F9001A59F37
:10288000300D1124F901E957FB4F6081E1817E2F62
:10289000777075956795FC01EE0FFF1FE55FFE4FA2
:1028A00071836083F901E857FB4FB081B695B69507
:1028B000B695E181FE2FF295FF0FF07E6F2F6B2B07
:1028C000E695E695E6957E2F777075956795FC0100
:1028D000EE0FFF1FE35FFE4F71836083F901E7573F
:1028E000FB4FB081B295B695B695B370C181DC2F20
:1028F000DD0FDD0F6D2F6B2BC295C695C695C3708E
:10290000E281E170EE0FEE0F7E2F7C2B75956795BF
:10291000FC01EE0FFF1FE15FFE4F71836083F90141
:10292000E557FB4FB081B695E181FE2FF795FF2764
:10293000F7956F2F6B2BE6957E2F777075956795C2
:10294000FC01EE0FFF1FEF5EFE4F71836083F90104
:10295000E457FB4FB081B295BF70E181FE2FF29535
:10296000F07F6F2F6B2BE295EF707E2F7770759550
:102970006795FC01EE0FFF1FED5EFE4F71836083D4
:10298000F901E357FB4FB081BB1FBB27BB1FC181C0
:10299000DC2FDD0F6D2F6B2BCC1FCC27CC1FE281E2
:1029A000E370EE0F7E2F7C2B75956795FC01EE0F83
:1029B000FF1FEB5EFE4F71836083F901E157FB4F10
:1029C000B081B695B695E181FE2FF295FF0FFF0F0E
:1029D000F07C6F2F6B2BE695E6957E2F77707595C3
:1029E0006795FC01EE0FFF1FE95EFE4F7183608368
:1029F000F901E057FB4F2081229526952770318100
:102A0000E32FEE0FEE0FEE0F6E2F622B732F7295EA
:102A10007695777075956795FC01EE0FFF1FE75E61
:102A2000FE4F718360834F5F5F4F4230510509F065
:102A30001ECF80919D0483FF1092A80410923C0445
:102A400080C0243009F07DC060913C0461110BC04E
:102A5000C83AB1F4109273051092720588EA0E9488
:102A6000610681E06CC0613019F4C093370404C082
:102A7000623031F4C09336048C2F0E9461065AC034
:102A8000E09136042E2F30E0220F331F462F50E006
:102A9000C9010296841795073CF0633268F7FA0182
:102AA000EC57FB4FC083E8CF2D5F3F4F8C2F90E05A
:102AB00060917205709173054217530749F4982F7E
:102AC000882786279727909373058093720532C0D5
:102AD0006817790769F580913704813049F5E1314C
:102AE00018F080E180933604F0903604C8E8D4E012
:102AF00000E010E00F15D0F4FE013197808190E0E6
:102B0000982F88272881822B43E0969587954A95B0
:102B1000E1F70E94DE08F801EE0FFF1FE55FFE4FB0
:102B2000918380830F5F1F4F2296E4CF1092A804F9
:102B300010923C0480913C04882319F08F5F8093AD
:102B40003C04CDB7DEB7E8E00C94022EE82FF0E0AD
:102B5000E854FA4FE185E03150F4F894F0E0EE0FDC
:102B6000FF1FE55FFE4F808191817894089580E09A
:102B700092E00895A2E2B0E0E0ECF5E10C94DC2DE7
:102B80009E012F5F3F4F80E1D9011D928A95E9F7A1
:102B900063E072E080EE95E029A33AA30E942F2A19
:102BA0000E947B0B1D8A1E8A1F8A188E312C212CB5
:102BB00000E0812C912C540170E4472E71EE572EC9
:102BC0007DE9672E78E1772EE0E5CE2EE3ECDE2E70
:102BD000E12CF12C84EF91E0A0E0B0E08D8F9E8F8E
:102BE000AF8FB8A380EC91EDA8E9BBE1898F9A8FF4
:102BF000AB8FBC8F80E491EEADE9B8E1898B9A8B05
:102C0000AB8BBC8B80EE95E00E94432B892B09F4A3
:102C1000E1C080EE95E00E94702B9C0133272C329E
:102C2000310509F442C0ACF42332310509F0ABC0E0
:102C300019821A821B821C821D821E821F821886A4
:102C400019861A861B861C861D861E861F86188A74
:102C500060C02434310529F02335310509F4B2C0B0
:102C600092C064E480EE95E00E94012A2AE030E000
:102C700040E451EE6DE978E180EE95E00E948F2A04
:102C80006CE280EE95E00E94012A2AE030E040EC00
:102C900051ED68E97BE180EE95E00E948F2A6CE2BD
:102CA00080EE95E00E94412AADCF0F5F043009F01D
:102CB000A9CF29813A814B815C81A8EEB3E00E94C3
:102CC000642D698B7A8B8B8B9C8B2D813E814F8100
:102CD00058850E94642D698F7A8F8B8F9C8F2985F0
:102CE0003A854B855C852D8F3E8F4F8F58A32D8560
:102CF0003E854F8558890E94642D6B017C016032AE
:102D00003EE473078105910530F462E38CE10E9493
:102D10009E0900E077CF603345E774078105910590
:102D200010F462E2F3CF60345CE975078105910528
:102D300010F466E2EBCF80E5C81683ECD806E10418
:102D4000F10410F462E1E2CF90E6C9169AEED906DA
:102D5000E104F10410F465E1D9CFA0E7CA16A1E1BE
:102D6000DA06A1E0EA06F10410F461E0CFCFB0EAA0
:102D7000CB16B6E8DB06B1E0EB06F10410F463E035
:102D8000C5CF65E0C3CF10ED180F1A3008F03ACF69
:102D9000E1E0F0E0EC0FFD1F24E0029FE00DF11DEB
:102DA00011242081318142815381AAE0B0E00E9448
:102DB000642D610F711D811D911D6083718382835C
:102DC000938320CF49885A886B887C88812C912CEA
:102DD000540118CF81149104A104B10489F4C301F2
:102DE000B2010E940D0A61E070E080E090E00E9474
:102DF00083281D8A1E8A1F8A188E312C22242A9429
:102E00008D8D9E8DAF8DB8A188169906AA06BB063A
:102E1000D0F40E94C7092D893E894F89588D280F0B
:102E2000311D411D511D2D8B3E8B4F8B588F3816F8
:102E300008F4382E821508F4282E3FEF831A930ADF
:102E4000A30AB30A56C0C301B20128EE33E040E042
:102E500050E00E949B2DBA01A9012AE030E080EEEB
:102E600095E00E94E62A6CE280EE95E00E94012A3D
:102E70004AE050E0632D80EE95E00E94F52A6CE276
:102E800080EE95E00E94012A6D897E898F89988D58
:102E9000A50194010E949B2DBA01A9012AE030E00E
:102EA00080EE95E00E94E62A6CE280EE95E00E94BA
:102EB000012A4AE050E0622D80EE95E00E94F52A5A
:102EC0006CE280EE95E00E94412A4C0C5D1C6E1C69
:102ED0007F1C898D9A8DAB8DBC8D84159505A605BB
:102EE000B70520F449885A886B887C88812C912CFE
:102EF000540129893A894B895C89283E3340410530
:102F0000510509F07FCEA296E2E10C94F82DACE1D8
:102F1000B0E0EDE8F7E10C94E62D0E9460286B012B
:102F20007C0181E00E947D0A14E703E0198361E0DF
:102F3000CE0101960E94DA0B009371050E94580B96
:102F40006AEF70E080E090E00E9483288091710534
:102F5000833089F480EE95E00E94432B892B59F44D
:102F60000E9460286C197D098E099F096038734C96
:102F7000894C9140D8F280917105833009F44FC09B
:102F80008FE70E9476090E9489098983843511F0B0
:102F900083E05CC00E948909109244058093450536
:102FA0000E9489092091440530914505280F311D63
:102FB00030934505209344050E9489098093460576
:102FC0000E94890980934705813110F7F12C0F2D5C
:102FD00010E08091470590E0880F991F08171907A6
:102FE00040F40E948909F801E85BFA4F8083F3946A
:102FF000EECF80E7898361E0CE0101960E94DA0B73
:1030000083E0809371050E94580B62E370E080E0DA
:1030100090E00E94832880917105833011F482E052
:1030200015C08FE70E9476090E948909898380353F
:1030300009F0AECF0DE915E00E948909F8018193EE
:103040008F01F5E0083B1F07B9F781E06C96E8E0D7
:103050000C94022E80914305992787FD9095A92F06
:10306000B92FFC013196EB30F10508F066C0EC5C3D
:10307000FF4F0C94132E62E778E080EE95E00E94FB
:103080001D2A80E893E00E942F0C6AE578E080EE2C
:1030900095E00E941D2A65E378E080EE95E00E94AD
:1030A0001D2A6BE078E080EE95E00E941D2A6AEE12
:1030B00077E080EE95E00E941D2A6DEB77E080EED0
:1030C00095E00E941D2A67E977E080EE95E00E9476
:1030D0001D2A63E777E080EE95E00E941D2A6CE4EC
:1030E00077E080EE95E00E941D2A80EE95E00E9438
:1030F000092A0E94600D21C06FE277E01AC06AE0E1
:1031000077E017C065EF76E014C066ED76E011C099
:1031100062E976E00EC06DE776E00BC068E676E027
:1031200080EE95E00E941D2A62E276E002C06CE02B
:1031300076E080EE95E00E941D2A6AE070E080E073
:1031400090E00E94832880EE95E00E94432B892B1B
:1031500029F080EE95E00E94702BF5CF0895ACE148
:10316000B0E0E5EBF8E10C94E62D909143059F3F2C
:1031700009F023C1482F50E0FA013A97EF36F105E4
:1031800008F00FC1E15CFF4F0C94132E60E172E078
:10319000A0C06CE172E080EE95E00E942F2A85E7E6
:1031A00089838BE1EDE9F5E0DE01129601900D9245
:1031B0008A95E1F76CE1CE0101960E94DA0B0E943C
:1031C000580B83E08093710568EC70E080E090E03C
:1031D0000E94832880917105843009F0E2C08FE756
:1031E0000E9476090E9489098983853509F0D9C032
:1031F0006DEE74E080EE95E00E941D2A6FEC74E0A5
:1032000080EE95E00E941D2A61EB74E096C064E3B5
:1032100072E080EE95E00E942F2A89E6898361E0C2
:10322000CE0101960E94DA0B0E94580B83E0809336
:10323000710568EC70E080E090E00E948328809146
:103240007105843009F0ADC08FE70E9476090E94B5
:10325000890989838E010E5F1F4F7E014DE1E40EC7
:10326000F11C0E948909F80181938F01EE15FF0579
:10327000C1F78BE1FE013296ADE9B5E001900D9208
:103280008A95E1F78981893409F08BC063E974E09C
:1032900080EE95E00E941D2A65E774E080EE95E0DF
:1032A0000E941D2A67E574E048C06EE472E080EE7B
:1032B00095E00E942F2A8EEF8093430572C08052C2
:1032C0008750805390914605981708F066C06DE5C9
:1032D00072E080EE95E00E942F2A63C084E1809323
:1032E000430560E274E029C085E18093430569EEFF
:1032F00073E023C086E18093430562EB73E01DC059
:1033000087E18093430568E673E017C088E1809306
:10331000430567E573E011C089E18093430563E4E9
:1033200073E00BC08AE1809343056EE273E005C051
:103330008BE18093430566E073E080EE95E00E94A8
:103340001D2A2FC06CEE72E080EE95E00E941D2ACF
:103350008091AB0591E01DC066ED72E080EE95E0D6
:103360000E941D2A8091AB0592E013C061EC72E0CF
:1033700080EE95E00E941D2A8091AB0594E009C083
:1033800066EA72E080EE95E00E941D2A8091AB050E
:1033900098E089278093AB058FEF809343050E94C7
:1033A000011080EE95E00E94432B892B09F45BC14C
:1033B00080EE95E00E94702BF4CF0E9400118823CC
:1033C00009F451C18091DD04811104C08FEF809315
:1033D000430541C140E050E060E070E08EED94E0D4
:1033E0000E948A2E40914305042F112707FD109556
:1033F000212F312FF8013197EB31F10508F01BC176
:10340000E255FF4F0C94132E552747FD5095209100
:10341000460530E0241735070CF40DC18B019C01E3
:103420000150110921093109003211052105310529
:1034300058F0C0904705E9E4F5E0F12CD12CA8E262
:10344000EA2E415051090FC0FA01E356FA4F61507C
:103450006083D9C0DF0111972C9130E02417350724
:1034600029F0F3943296FC10F5CFCBC00E2D10E06E
:1034700020E030E0061717072807390741F42081BC
:10348000DA01A356BA4F11962C93DD24D394E3941A
:10349000E8CF6F3F71058105910511F008F0CBC0B1
:1034A0006093B505B0C06F3F71058105910511F0BE
:1034B00008F0C1C06093B605A6C06F3F71058105D5
:1034C000910511F008F0B7C06093B7059CC020913A
:1034D000DE0420622037E9F440E050E060E070E074
:1034E0008FED94E00E948A2E9B01AC01DC01CB01A0
:1034F0000197A109B1090897A105B10508F0AEC06F
:10350000A4EDB0E30E94642D6A5E7C4A8A46954E23
:1035100024C02636E9F440E050E060E070E08FED32
:1035200094E00E948A2E9B01AC01DC01CB01019743
:10353000A109B1090797A105B10508F08FC0A8EA54
:10354000B1E60E94642D645E7C438E46944E05C0B5
:10355000611571058105910579F08B019C0100547D
:10356000114E2D4938410138F0EF1F07FAEF2F07B0
:10357000F2E03F0708F05FC06093AD057093AE05C1
:103580008093AF059093B0053EC06F3F71058105F4
:10359000910511F008F04FC06093B10534C08B0164
:1035A0009C0101501109210931090F3F1105210525
:1035B000310508F040C06093B20525C08B019C0125
:1035C000045C1940210931090D344DE1140721052E
:1035D000310528F47093B4056093B30514C06115E8
:1035E00071058105910521F48FEF8093AC050BC027
:1035F0006134710581059105F0F461506093AC056B
:1036000002C0DD20C1F08091DC0481111AC08091DC
:103610007D0590917E05A0917F05B0918005019672
:10362000A11DB11D80937D0590937E05A0937F051C
:10363000B093800506C06FE672E080EE95E00E94D0
:103640002F2A0E94F6108FEF809343056AE080EEE8
:1036500095E00E94412A0E94011005C061E070E0DF
:1036600080E090E07ACF6C96E8E00C94022E6AE558
:1036700072E080EE95E00E941D2A62E472E080EE26
:1036800095E00E941D2A80EE95E00E94432B892B35
:1036900031F080EE95E00E94702B0E94AF180E94DE
:1036A0008717823029F0833051F46DE072E002C058
:1036B00064E272E080EE95E00E941D2A08958FEF8B
:1036C000809343051092DC040E9401108091430511
:1036D0008E3F69F080EE95E00E94432B892BB1F379
:1036E00080EE95E00E94702B0E94AF18EFCF0895F6
:1036F0000F931F93109143051F3F09F0D2C08934E7
:1037000009F457C000F5883309F469C058F48033D0
:1037100009F477C008F061C08B3109F440C08132F0
:10372000B1F1B9C0813409F487C030F4893309F4A8
:1037300066C0803461F1AFC0823409F48EC0863433
:1037400009F448C0A8C0823609F487C078F48835E7
:1037500031F128F48235C1F18335E1F09CC08A351E
:1037600009F494C0813609F467C095C0823761F1CD
:1037700028F4863679F18936E1F08DC0883779F002
:103780008A3709F483C0833709F085C003C060E13C
:1037900072E015C00E94310D6DE872E004C00E9415
:1037A0003A0D67EA72E080EE95E00E942F2A8EEFD4
:1037B00070C00E947A060E94BF0666EC72E080EE3E
:1037C00095E00E942F2A67C081E00E94DF066FED1E
:1037D00072E0F5CF0E94AB105EC080535AC06AEF12
:1037E00071E080EE95E00E941D2A90919C0588E092
:1037F000890F8871977E892B80939C051AC089E078
:1038000048C067EE71E080EE95E00E941D2A80912D
:10381000BD059091BE05A091BF05B091C00520E106
:1038200082278093BD059093BE05A093BF05B093FA
:10383000C005109343052FC061ED71E080EE95E067
:103840000E941D2A8091BD059091BE05A091BF05E3
:10385000B091C00540E4842710C060EC71E080EEB8
:1038600095E00E941D2A8091BD059091BE05A09112
:10387000BF05B091C00520E282278093BD059093DB
:10388000BE05A093BF05B093C00502C00E94371BC0
:103890008FEF80934305809143058E3F09F0D4C09C
:1038A000DDC00E940011882309F4D8C08091DD0496
:1038B000811104C08FEF80934305C6C040E050E003
:1038C00060E070E08EED94E00E948A2E0091430546
:1038D000112707FD1095212F312FF8013197E9307D
:1038E000F10508F0B4C0E753FF4F0C94132E8B0181
:1038F0009C010154114E2D4938410F37104F2A4F6A
:10390000324008F0A4C06093790570937A058093E3
:103910007B0590937C0577C060937D0570937E0551
:1039200080937F059093800581E08093DC046BC0D9
:10393000683071058105910508F089C060938105A3
:1039400062C08B019C0101501109210931090A3023
:1039500011052105310508F07AC06093820553C036
:1039600060EB71E08EED94E00E94C42F10E00097B0
:1039700099F00E949E2F009779F0183130F4E12FD2
:10398000F0E0EC58FA4F87871F5F60EB71E080E052
:1039900090E00E94C42FEBCF1831A8F5E12FF0E0A2
:1039A000EC58FA4F17861F5FF7CF65307105810518
:1039B000910508F04CC060939B0525C08B019C01CC
:1039C0000150110921093109063011052105310580
:1039D000F0F520919C05287F262B20939C0513C091
:1039E0008B019C0101501109210931090115124C6B
:1039F0002140310560F560937505709376058093DD
:103A00007705909378058091DC04811113C0809133
:103A10007D0590917E05A0917F05B091800501966E
:103A2000A11DB11D80937D0590937E05A0937F0518
:103A3000B09380050E94F6108FEF809343056AE0F3
:103A400080EE95E00E94412A0E942A1807C06FE686
:103A500072E080EE95E00E942F2AECCF1F910F912B
:103A600008958FEF809343051092DC040E942A187A
:103A7000809143058E3F69F080EE95E00E94432BD4
:103A8000892BB1F380EE95E00E94702B0E94781B89
:103A9000EFCF6AE070E080E090E00E94832880EE43
:103AA00095E00E94432B892B29F080EE95E00E943F
:103AB000702BF5CF0895CF93C82F682F80EE95E037
:103AC0000E949D2B909168059C2790936805CF914B
:103AD0000895A1E0B0E0EFE6FDE10C94EC2D9983B0
:103AE0000E945B1D9981892F0E945B1D2196E2E057
:103AF0000C94082E1F93CF93DF93182FEB01109295
:103B0000680565EB70E080EE95E00E94590662E67C
:103B100070E080EE95E00E945906812F0E945B1DA7
:103B2000CE010E94691DDF91CF911F910895609190
:103B3000680580EE95E00E949D2B0895A1E2B0E01B
:103B4000E4EAFDE10C94E82D7B018A018C3009F454
:103B500052C108F040C0863009F4BCC018F583306B
:103B600009F491C070F4813009F472C0823009F018
:103B700047C26BE170E082E00E947A1D0DE915E01A
:103B800078C0843009F487C0853009F039C260916B
:103B9000470570E0660F771F85E00E947A1D08E4F4
:103BA00015E086C0893009F4A7C070F4873009F4A5
:103BB0009BC0883009F024C261E070E088E00E9478
:103BC0007A1D8091D20522C28A3009F4CAC08B3096
:103BD00009F4F1C015C28A3609F474C1D8F48736E5
:103BE00009F439C138F4853609F40DC1863609F473
:103BF0001EC106C2883609F436C1893609F000C2F2
:103C000061E070E089E60E947A1D0E947A060E94B7
:103C1000BF06F4C18D3609F4D3C138F48B3609F4EC
:103C200090C18C3609F499C1EBC18E3609F4DBC121
:103C3000873C09F0E5C161E070E087EC0E947A1DE5
:103C400081E00E945B1D0E94971D10926905E2C1F0
:103C500069E270E081E00E947A1D04E715E0F80156
:103C600081918F010E945B1DF5E00D391F07B9F7A7
:103C7000CFC1F80181918F010E945B1DF5E0083BE7
:103C80001F07B9F7C5C161E070E083E00E947A1DAB
:103C90000E948717BBC161E070E084E00E947A1D3A
:103CA00081E00E945B1D0E94971D0E94BA15B2C15F
:103CB0008091470590E0880F991F9801285435405E
:103CC0002817390708F0A4C1F80181918F010E94DB
:103CD0005B1DEECF62E070E086E00E947A1D80E816
:103CE00093E00E94691D94C161E070E087E00E944A
:103CF0007A1D809146058AC186E6898361E0CE01FE
:103D000001960E94DA0B0E94580B83E080937105A4
:103D100068EC70E080E090E00E948328809171055B
:103D20008430D9F48FE70E9476090E94890989833B
:103D3000863469F460E270E089E00E947A1D10E246
:103D40000E9489090E945B1D1150D1F761C161E099
:103D500070E089E00E947A1D51C161E070E089E065
:103D600052C169E170E08AE00E947A1D1092B805A4
:103D7000209170058091BD059091BE05A091BF0571
:103D8000B091C005222311F0806801C08F77809325
:103D9000BD059093BE05A093BF05B093C00508EB89
:103DA00015E0F80181918F010E945B1DF5E0013D56
:103DB0001F07B9F72DC161E270E08BE00E947A1D08
:103DC0008091A8048F3F39F08091A80491E0980F6A
:103DD0009093A80402C08091A8040E945B1D10E08B
:103DE000812F0E94A6150E9409090E94691D1F5F6C
:103DF0001031B1F70DC161E070E08CE00E947A1DD6
:103E00008091D10503C161E070E085E60E947A1DD2
:103E100089E2E816F10409F0F8C0D801E4E7F5E01A
:103E20008D91819385E0ED39F807D1F7E7C061E026
:103E300070E086E60E947A1DEBE1EE16F10409F0CF
:103E4000E4C0D801EDE9F5E08D91819385E0E83B90
:103E5000F807D1F7D3C061E070E087E60E947A1DD1
:103E60000E94310DCBC061E070E088E60E947A1DAF
:103E700085E789838BE1EDE9F5E0DE01129601909B
:103E80000D928A95E1F76CE1CE0101960E94DA0B62
:103E90000E94580B83E08093710560E273E080E03C
:103EA00090E00E94832880917105843009F0ADC0B4
:103EB0008FE70E9476090E9489098983853509F078
:103EC000A4C09CC061E070E08AE60E947A1D89E689
:103ED000898361E0CE0101960E94DA0B0E94580BA3
:103EE00083E08093710560E273E080E090E00E94DF
:103EF000832880917105843009F087C08FE70E9484
:103F000076090E94890989838E010E5F1F4F7E0109
:103F1000EDE1EE0EF11C0E948909F80181938F01F9
:103F2000EE15FF05C1F78BE1FE013296ADE9B5E074
:103F300001900D928A95E1F78981893409F065C075
:103F40005DC061E070E08BE60E947A1DF80180811F
:103F50008093D2050E943A0D51C061E070E08CE67A
:103F60000E947A1DF0E2EF16F10461F487E689837E
:103F700080E2F801DE01129601900D928A95E1F738
:103F800061E203C087E4898361E0CE0101960E946B
:103F9000DA0B0E94580B83E0809371056CE474E0A7
:103FA00080E090E00E94832880917105843069F55B
:103FB0008FE70E9476090E948909873431F51EC077
:103FC00061E070E08DE60E947A1D89E1E816F10457
:103FD000E1F4D801E8EBF5E08D91819385E0E13DD6
:103FE000F807D1F70BC061E070E08EE60E947A1D01
:103FF000F80180818093D1050E941A0D81E006C0EE
:1040000061E070E08AEC0E947A1D80E00E945B1DF6
:104010000E94971DA196E6E00C94042EA0E0B0E06B
:10402000E4E1F0E20C94E62DCAECD3E014E606E0FD
:1040300035E0F32E44E0E42E53E0D52E62E0C62EA8
:1040400080EE95E00E94432B892B09F49BC080EE03
:1040500095E00E94702B282F809335044091340402
:1040600050E04730510560F7FA01EE52FF4F0C94D3
:10407000132E853B29F781E080933404E1CF82360B
:1040800009F07DC0C0923404DBCF80933304809369
:104090003204D0923404D4CF9C01332730933104BE
:1040A0002093300490913204982790933204E09248
:1040B0003404C6CF382F2227409130045091310468
:1040C000242B352B3093310420933004909132040B
:1040D000982790933204F09234042536310508F481
:1040E000AFCF61E070E08CEC0E947A1D81E00E940D
:1040F0005B1D0E94971D43C020912E0430912F0418
:10410000F901E653FC4F80839091320498279093F5
:104110003204C901019690932F0480932E042091BC
:104120003004309131048217930708F489CF00934B
:10413000340486CF8091320482130BC060912E0428
:1041400070912F044AEC53E0809133040E949E1D2D
:104150000DC062E070E08BEC0E947A1D8091330408
:104160000E945B1D809168050E945B1DFE01812FEE
:1041700011928A95E9F710922F0410922E04109252
:1041800034045ECFCDB7DEB7E8E00C94022E81E0B8
:104190008093690580916905882349F080EE95E058
:1041A0000E94432B892BB1F30E940E20F3CF089578
:1041B000AAE2B0E0EEEDF0E20C94E42D0E94542867
:1041C0006B017C0181E00E947D0A80EE95E00E94F7
:1041D000432B892B29F080EE95E00E94702BF5CFC0
:1041E0002C9811E072E6B72EE9E2AE2E03E00E94B1
:1041F00054286C197D098E099F09693C7105810558
:104200009105D0F11123C1F10E9454286B017C016A
:104210002B9A80ED97E00E94A807B982E4E7F5E0C9
:10422000DE0112968A2D01900D928A95E1F76AE2DD
:10423000CE0101960E94DA0B2B9880E090E00E945C
:10424000A807009371050E94580B62E370E080E0BC
:1042500090E00E94832880917105843061F400937E
:1042600071058FE70E9476090E94890911E0823466
:1042700019F410E001C011E08AE00E947929892B2D
:1042800081F411E00EC02C9A2B9A80EE95E00E94EA
:10429000702B8D309105A9F05CF40A9791F02C9861
:1042A0002B9880EE95E00E94432B892B61F79FCFDE
:1042B0008332910579F08234910589F70E94C720F5
:1042C000EECF62EB71E080EE95E00E941D2A0E9425
:1042D000311DE5CF0E94BA15E2CF8F929F92AF9227
:1042E000BF92CF92DF92EF92FF921F93CF93DF9313
:1042F0008AE00E947929892B09F089C068EC70E076
:1043000080E090E00E94832880E090E00E94A8076F
:104310000E9454284B015C016B017C0180ECC80EAB
:1043200082E1D81EE11CF11C0E9454286C157D0509
:104330008E059F0530F48AE00E947929892BA1F32C
:1043400064C08AE00E947929892B09F05EC080ED63
:1043500097E00E94A8070E9454286B017C01D0E0DE
:10436000C1E088E4880E86E2981EA11CB11C11E011
:104370008AE00E947929892B21F58C149D04AE04D2
:10438000BF0430F480ED97E00E94A807D1E0F0CFA1
:104390000E9454286C197D098E099F09693C71059A
:1043A0008105910528F30E9454286B017C01C127E7
:1043B00019F080ED97E002C080E090E00E94A8072D
:1043C000D7CF80E090E00E94A807DD23B9F080916C
:1043D000D10590E0019665E070E00E94872D809302
:1043E000D1050E941A0D0E949B130E943A0D64EFA2
:1043F00071E080E090E00E94832809C080E00E9484
:10440000DF060E94B2110E94310D0E94D820DF9178
:10441000CF911F91FF90EF90DF90CF90BF90AF9022
:104420009F908F900895CF92DF92EF92FF9280E05D
:104430000E94DA070E94B10761E08CE00E940D291A
:1044400061E08BE00E940D2960E08AE00E940D2966
:1044500060E083E10E940D2961E083E10E9446292A
:1044600061E082E10E940D2960E082E10E9446291C
:104470000E949F0740E052EC61E070E080EE95E022
:104480000E948B2C0E949B130E943A0D0E94841361
:104490008FEF8093A8040E94C60778940E94542846
:1044A0006B017C018091A8048F3F59F40E9454282D
:1044B0006C197D098E099F09603D77408105910542
:1044C00088F380ED97E00E94A80761E08AE00E94EF
:1044D00046292C9A80EE95E00E94432B892B29F0E7
:1044E00080EE95E00E94702BF5CF6CEF72E080EECD
:1044F00095E00E94FE2980E893E00E942F0C63E182
:1045000073E080EE95E00E94FE294AE050E060E012
:1045100070E080EE95E00E94CE2A62E370E080E0D9
:1045200090E00E94832880EE95E00E94432B049740
:104530000CF180EE95E00E94702B82349105D1F44D
:1045400080EE95E00E94702B8E34910599F480EEF8
:1045500095E00E94702B8434910561F480EE95E023
:104560000E94702B819731F480E090E00E94A807B0
:104570000E94D8204091750550917605609177058D
:1045800070917805DB01CA010197A109B10904976F
:10459000A105B10568F44093A704433029F440EA2B
:1045A00056E861E070E004C040E052EC61E070E089
:1045B00080EE95E00E948B2C0E946D212C9880E06B
:1045C00090E00E94A8070E9484131092C304809177
:1045D000BD0583FF11C080918905882351F080912A
:1045E0009005882331F080919705882311F087E0AA
:1045F00001C085E08093C30480E00E947D0A809121
:10460000C4040E94B1090E94580B10923F041092FA
:104610003E0410923D04F12C8091D2058F15B0F02C
:1046200062E370E080E090E00E94832880ED97E0F4
:104630000E94A80762E370E080E090E00E94832877
:1046400080E090E00E94A807F394E6CF80919C055B
:1046500084FF08C0982F987181E0983109F080E0BC
:104660000E946E118FE00E94DA07FF90EF90DF90BA
:10467000CF900895EF92FF920F931F93CF93DF9304
:104680008C016EE770E080EE95E00E945906E8012B
:10469000F12CF0E2EF2E8E0188818D57823048F4A4
:1046A0006DE770E080EE95E00E94590688818E25C6
:1046B00088832196F801608180EE95E00E949D2B11
:1046C000F394F9E0FF12E7CF6EE770E080EE95E03B
:1046D0000E945906CDB7DEB7E6E00C94042EA9E09F
:1046E000B0E0E5E7F3E20C94EC2D9091C504911154
:1046F0000EC09EEF99838A836B8350E05595479552
:104700004C832D83198618861F821E822EC04091ED
:10471000CA04842F90E0B4E095958795BA95E1F7A7
:10472000242F2F7030E08217930719F18DEF8983C2
:104730001B82FE01349650E0842F90E0A4E0959512
:104740008795AA95E1F7242F2F7030E08217930701
:1047500049F0DC01A553BB4F8C918193405F5F5FB3
:10476000563051F74093CA045A83CE0101960E94F5
:104770003A238091C50490E0019666E070E00E94C3
:10478000872D8093C5042996E2E00C94082EA0E0C2
:10479000B0E0EDECF3E20C94E52D6C016EE770E017
:1047A00080EE95E00E9459068601E12CF12CC0E0D4
:1047B000D0E030E2B32EF801608183E8860F8230CA
:1047C00078F46DE770E080EE95E00E945906F801FC
:1047D00060816B2570E080EE95E00E94590604C070
:1047E00080EE95E00E949D2BE114F10459F0F80150
:1047F00080819E01280F311DC901C92FDD27C80FF7
:10480000D91FDD273FEFE31AF30A89E0E816F10428
:1048100059F028E0E216F10421F48C2F8095F6017E
:1048200080870F5F1F4FC7CFCDB7DEB7E9E00C948D
:10483000012EA9E0B0E0EFE1F4E20C94EC2DE82FBA
:10484000362F8091C50490E0019664E270E00E94EA
:10485000872D8093C50458E9598350E15A838130EC
:1048600089F048F08230B9F08330D9F48B8381EF3E
:104870008C833D8319C085E08B8381EF8C832F5F10
:104880002D8312C08B8381EF8C8384E6489FA00127
:1048900011245D8309C084E08B8381EF8C83ED83D9
:1048A00003C00E94AB1104C0CE0101960E94C72331
:1048B0002996E2E00C94082EA2E0B0E0E2E6F4E2F1
:1048C0000C94E12D182F762E2A8349830E946028AC
:1048D0006B017C018091DB048090C6049090C7043A
:1048E000A090C804B090C9042A8149818823C1F0EE
:1048F000D701C60188199909AA09BB094C015D01B4
:1049000091EE89169EE29906A104B10420F12417C4
:1049100008F4422F202F672D812F0E94192413C0E5
:10492000D701C60188199909AA09BB094C015D0183
:1049300091E3891695E79906A104B10460F0672D0B
:10494000812F0E946F23C092C604D092C704E092C8
:10495000C804F092C9042296EDE00C94FD2DA2E269
:10496000B0E0E5EBF4E20C94E22D8CE00E949809B3
:1049700081110DC06BE173E080EE95E00E942F2A5B
:104980002C9A80E00E947D0A0E94580B2C9880EEA1
:1049900095E00E94432B892B01F180EE95E00E9467
:1049A000702B9091A704992319F00E94AE13EFCFBA
:1049B00040913E0450E09A012F5F3F4F2F71332703
:1049C00060913F0470E02617370709F3FA01E75BAF
:1049D000FB4F808320933E04DACF809171058430B1
:1049E00009F086C00E946028611571058105910556
:1049F00049F06093B5047093B6048093B704909324
:104A0000B8040CC081E090E0A0E0B0E08093B50471
:104A10009093B604A093B704B093B8048091AB040C
:104A20009091AC0481609093AC048093AB0483E0DC
:104A3000809371058FE70E94760909E614E00E94D1
:104A40008909F80181938F01F4E002371F07B9F754
:104A50002091720480916904982F922796FF3BC0A1
:104A600090E4922790937204982F98739833F1F4FE
:104A700010E0212F30E080916904877090E0821768
:104A800093074CF11F5F20919C05812F90E0FC0162
:104A9000E759FB4F24FF04C080810E948D11E9CFAC
:104AA000608180EE95E00E949D2BE3CF8F7399F497
:104AB00080916A048093B40480916B048093B20463
:104AC00080916C048093B10480916F0490E0909386
:104AD000AA048093A90480913D04813019F482E0F6
:104AE00080933D0480913D04833011F410923D0485
:104AF0000E9460286B017C018091AD049091AE040E
:104B0000A091AF04B091B0040097A105B105C9F020
:104B1000A7019601281B390B4A0B5B0BDA01C9016F
:104B2000883B9B40A105B10560F00E94C7098093B6
:104B3000B3041092AD041092AE041092AF04109220
:104B4000B0048091B9049091BA04A091BB04B091D3
:104B5000BC0446015701881A990AAA0ABB0A84E7CD
:104B600095E00E94F40786169706A806B90608F491
:104B7000A8C0C092B904D092BA04E092BB04F092EB
:104B8000BC040E9457068091A8048830A0F0809150
:104B9000BD059091BE05A091BF05B091C0056CE127
:104BA000B695A795979587956A95D1F7892B8A2B06
:104BB0008B2B09F0A4C18091A8048F5F8093A80477
:104BC0008091B5049091B604A091B704B091B80457
:104BD0000097A105B105F1F0C81AD90AEA0AFB0A43
:104BE00084E795E00E94F4076C157D058E059F050E
:104BF00008F006C18091BD0584FD04C080ED97E0FA
:104C00000E94A8071092B5041092B6041092B7043F
:104C10001092B80490917204907C90937204509119
:104C20003E0480913F0420913D04581709F405C1CA
:104C3000223009F002C1905890937204E0919C05D3
:104C4000E770F0E0E758FC4F6081693008F0DDC0A4
:104C5000615040E04613DBC080933F0487E3840F3C
:104C600090917204892B809372044093400483E0F6
:104C700080933D042B9A809181059091C3049111FA
:104C80002FC10E94780A8091C4040E94B109E0916A
:104C90009C05E770F0E0E758FC4F608182E794E004
:104CA0000E94930BE091C404EF5FE093C404E831E9
:104CB00009F422C1F0E0EC58FA4F8785882309F403
:104CC0001BC10E94020C813069F580919C0588719E
:104CD00049F18091AB049091AC04880F991F909397
:104CE000AC048093AB0483E0809371050E94580B61
:104CF0000E9460286093AD047093AE048093AF046B
:104D00009093B004672B682B692B61F481E090E0ED
:104D1000A0E0B0E08093AD049093AE04A093AF0404
:104D2000B093B00480919C0584FF1FC08091AB04B8
:104D30009091AC048E7F0E942A09182F6091A904DB
:104D40008091B4040E94A413482F612F8091B30472
:104D500049A30E94A4130091D205282F49A1609174
:104D6000B1048091B2040E945C242B988091C1040C
:104D70008130C1F018F08230B1F1CEC08AE00E94DB
:104D80007929892B09F0C8C081E08093C1040E9471
:104D900054286093BD047093BE048093BF04909325
:104DA000C004BAC08AE00E947929892B31F50E949B
:104DB0005428C090BD04D090BE04E090BF04F09091
:104DC000C0046C197D098E099F09693E73408105F5
:104DD000910508F4A1C082E08093C10480ED97E0C2
:104DE0000E94A80799C08AE00E947929892B09F4BA
:104DF00093C080E090E00E94A8071092C1048CC08C
:104E000080E090E00E94A80705CF68E022CF8517D8
:104E100009F422CF4F5F242F30E090E0F901EE58E3
:104E2000FB4FDC01A75BBB4F7C917083F901E05C19
:104E3000FB4F708301968F710DCF2430B1F4209118
:104E4000400481E494E0A3E7B4E0FC013E2F381B6A
:104E5000321718F431913D93F9CF87E3820F909187
:104E60007204892B8093720402CF8091C104823036
:104E700069F49160909372042C9A51ECE52E55E000
:104E8000F52E8E010F5F1F4FB80110C02C98809136
:104E90003D04811103C081E080933D0480913D0475
:104EA000833059F784E080933D04E7CFF701819187
:104EB0007F0169A37AA30E94A615F80181939193BB
:104EC0008F0169A17AA1F1EDEF16F5E0FF0671F708
:104ED00080919C0543E754E087700E947908CACE10
:104EE000882309F4CECE2091C20431E0320F3093F2
:104EF000C2042913C6CE0CC01092C404E2CE809125
:104F0000A804883009F42C9A89E08093A804D9CEAB
:104F10001092C2048150B5CEA296ECE00C94FE2D06
:104F20008230E8F4E82FF0E0EE0FFF1FED52FA4F69
:104F300071836083813041F0809169008C7F842B84
:104F400080936900E89A089580916900440F551F85
:104F5000440F551F837F842B80936900E99A08953D
:104F60001F920F920FB60F9211242F933F934F93DE
:104F70005F936F937F938F939F93AF93BF93EF93C1
:104F8000FF938091D3059091D405892B29F0E0916E
:104F9000D305F091D4050995FF91EF91BF91AF91A1
:104FA0009F918F917F916F915F914F913F912F9141
:104FB0000F900FBE0F901F9018951F920F920FB673
:104FC0000F9211242F933F934F935F936F937F938F
:104FD0008F939F93AF93BF93EF93FF938091D505EA
:104FE0009091D605892B29F0E091D505F091D60551
:104FF0000995FF91EF91BF91AF919F918F917F9113
:105000006F915F914F913F912F910F900FBE0F9035
:105010001F9018951F920F920FB60F9211242F9385
:105020003F938F939F93AF93BF938091D8059091B7
:10503000D905A091DA05B091DB053091D70523E0C1
:10504000230F2D3720F40196A11DB11D05C026E8C0
:10505000230F0296A11DB11D2093D7058093D8057B
:105060009093D905A093DA05B093DB058091DC0518
:105070009091DD05A091DE05B091DF050196A11D9F
:10508000B11D8093DC059093DD05A093DE05B09300
:10509000DF05BF91AF919F918F913F912F910F901D
:1050A0000FBE0F901F9018952FB7F8946091D805F8
:1050B0007091D9058091DA059091DB052FBF089595
:1050C0003FB7F8948091DC059091DD05A091DE0555
:1050D000B091DF0526B5A89B05C02F3F19F00196BA
:1050E000A11DB11D3FBF6627782F892F9A2F620F10
:1050F000711D811D911D42E0660F771F881F991F4A
:105100004A95D1F70895CF92DF92EF92FF92CF9315
:10511000DF936B017C010E946028EB01C114D10474
:10512000E104F10479F00E9460286C1B7D0B683E5D
:105130007340A0F381E0C81AD108E108F108C85112
:10514000DC4FECCFDF91CF91FF90EF90DF90CF90CD
:105150000895789484B5826084BD84B5816084BDEF
:1051600085B5826085BD85B5816085BDEEE6F0E0E0
:10517000808181608083E1E8F0E01082808182603C
:105180008083808181608083E0E8F0E080818160BD
:105190008083E1EBF0E0808184608083E0EBF0E0ED
:1051A000808181608083EAE7F0E080818460808391
:1051B000808182608083808181608083808180683B
:1051C00080831092C1000895833081F028F48130EB
:1051D00099F08230A1F008958630A9F08730B9F0B7
:1051E0008430D1F4809180008F7D03C08091800055
:1051F0008F7780938000089584B58F7702C084B53F
:105200008F7D84BD08958091B0008F7703C0809119
:10521000B0008F7D8093B0000895CF93DF9390E02E
:10522000FC01ED50F44F2491FC01E95FF34F8491B0
:10523000882349F190E0880F991FFC01E15DF34F4D
:10524000A591B4918B5D934FFC01C591D4919FB70B
:10525000611108C0F8948C91209582238C938881E9
:1052600082230AC0623051F4F8948C91322F309529
:1052700083238C938881822B888304C0F8948C913B
:10528000822B8C939FBFDF91CF910895A1E0B0E076
:10529000ECE4F9E20C94EA2D282F30E0F901E15218
:1052A000F44F8491F901ED50F44F1491F901E95F45
:1052B000F34F04910023C9F0882321F069830E94F1
:1052C000E4286981E02FF0E0EE0FFF1FEB5DF34F64
:1052D000A591B4919FB7F8948C91611103C010957A
:1052E000812301C0812B8C939FBF2196E4E00C9415
:1052F000062ECF93DF93282F30E0F901E152F44FCF
:105300008491F901ED50F44FD491F901E95FF34F25
:10531000C491CC2391F081110E94E428EC2FF0E09D
:10532000EE0FFF1FE55EF34FA591B4912C912D2355
:1053300081E090E021F480E002C080E090E0DF9125
:10534000CF910895A0E0B0E0E8EAF9E20C94E62DF0
:105350006C017A01EB01E60EF71E00E010E0CE15BD
:10536000DF0561F06991D601ED91FC910190F0812A
:10537000E02DC6010995080F191FF1CFC801CDB75F
:10538000DEB7E8E00C94022E6115710589F0DB01AF
:105390000D900020E9F7AD0141505109461B570B14
:1053A000DC01ED91FC910280F381E02D09950895D7
:1053B00080E090E00895EF92FF920F931F93CF93B8
:1053C000DF938C01FB01C0E0D0E064917F018FEF9F
:1053D000E81AF80A662361F0D801ED91FC9101907A
:1053E000F081E02DC8010995C80FD91FF701EDCF55
:1053F000CE01CDB7DEB7E6E00C94042E0E94C4299E
:105400000895DC01ED91FC910190F081E02D09956A
:1054100008950F931F93CF93DF93EC016DE00E94EB
:10542000012A8C016AE0CE010E94012A800F911F9F
:10543000DF91CF911F910F9108950F931F93CF93F9
:10544000DF93EC010E94DB298C01CE010E94092A26
:10545000800F911FDF91CF911F910F9108950F93AE
:105460001F93CF93DF93EC010E94C4298C01CE01DE
:105470000E94092A800F911FDF91CF911F910F91F8
:1054800008950F931F93CF93DF93EC010E94012A9D
:105490008C01CE010E94092A800F911FDF91CF91CC
:1054A0001F910F910895A1E2B0E0E9E5FAE20C94B2
:1054B000E22D7C01C42EE52FCB01D22E19A221E0D2
:1054C0002D1510F02AE0D22E8E010F5D1F4F8D2C6E
:1054D000912CA12CB12C6C2D7E2FA50194010E9442
:1054E0009B2D8C2DD29E80191124015011098A30D8
:1054F00010F4805D01C0895CF801808321153105BD
:105500004105510521F0C22EE32FCA01E4CFB801B5
:10551000C7010E94C429A196ECE00C94FE2DA0E0E6
:10552000B0E0E5E9FAE20C94E62DEC016A017B01BA
:105530002115310541F4E881F9810190F081E02DD8
:10554000642F09951DC02A303105A9F477FF12C0D8
:105550006DE20E94012A8C0144275527BA014C199B
:105560005D096E097F092AE0CE010E94532A800F4F
:10557000911F06C02AE0B701A601CE010E94532A5E
:10558000CDB7DEB7E8E00C94022E9A01AB01662796
:1055900057FD6095762F0E948F2A08950F931F93D1
:1055A000CF93DF93EC019A01AB01662757FD60951D
:1055B000762F0E948F2A8C01CE010E94092A800F2B
:1055C000911FDF91CF911F910F9108952115310502
:1055D00049F4DC01ED91FC910190F081E02D642F04
:1055E000099508950E94532A08959A01462F50E084
:1055F00060E070E00E94E62A08959A01AB0160E045
:1056000070E00E94E62A08950F931F93CF93DF93D3
:10561000EC010E94E62A8C01CE010E94092A800F2B
:10562000911FDF91CF911F910F9108950F931F93B9
:10563000CF93DF93EC019A01AB0160E070E00E9430
:10564000E62A8C01CE010E94092A800F911FDF916A
:10565000CF911F910F9108950F931F93CF93DF93D5
:10566000EC019A01462F50E060E070E00E94E62ACB
:105670008C01CE010E94092A800F911FDF91CF91EA
:105680001F910F910895FC0124853585F901E05C97
:10569000FF4F80819181F901EE5BFF4F20813181C5
:1056A000821B930B8F7399270895FC018485958540
:1056B000FC01E05CFF4F40815181FC01EE5BFF4F3C
:1056C000208131814217530741F00190F081E02D94
:1056D000E80FF91F808190E008958FEF9FEF089504
:1056E000FC0184859585FC01E05CFF4F4081518180
:1056F000FC01EE5BFF4F208131814217530779F0A7
:10570000A081B181A80FB91F8C91208131812F5FB9
:105710003F4F2F7333273183208390E008958FEF1D
:105720009FEF0895FC0181A1882329F0A489B58900
:105730008C9186FFFBCF11A20895CF93DF93FC01DC
:1057400026853785D901A05CBF4F8D919C9111971B
:1057500001968F739927E901CE5BDF4F488159810C
:1057600084179507D9F30D90BC91A02DA20FB31FFC
:105770006C93A685B785A05CBF4F11969C938E93C2
:10578000A689B7892C9181E090E0078C02C0880F30
:10579000991F0A94E2F7282B2C9381E081A30488B7
:1057A000F589E02D80818064808381E090E0DF9145
:1057B000CF91089508951F920F920FB60F92112462
:1057C0002F933F934F938F939F93EF93FF938091EA
:1057D000C00082FD1CC04091C60080918606909159
:1057E000870601968F739927209188063091890644
:1057F0008217930771F0E0918606F0918706EA5BC5
:10580000F94F4083909387068093860602C080916B
:10581000C600FF91EF919F918F914F913F912F91F2
:105820000F900FBE0F901F90189580EE95E00E948C
:10583000432B892B11F00E94DA2B08951F920F92AF
:105840000FB60F9211242F933F938F939F93EF9353
:10585000FF93209142063091430680914406909137
:1058600045062817390731F48091C1008F7D809358
:10587000C10014C0E0914406F0914506EE5FF94F77
:105880002081809144069091450601968F73992757
:1058900090934506809344062093C600FF91EF91B4
:1058A0009F918F913F912F910F900FBE0F901F905E
:1058B0001895A0E0B0E0EFE5FCE20C94E22DFC01CD
:1058C0001382128288EE93E0A0E0B0E08483958397
:1058D000A683B7838BEB93E091838083758764877E
:1058E00057874687318B208B138B028BF58AE48A8E
:1058F000D78AC68AB18EA08E938E828E8F85848F32
:105900008889858F8989868F8A89878F8B8980A3EB
:10591000ECE00C94FE2DCF92DF92EF92FF92CF93AA
:10592000DF93EC016A017B01411581EE58076105A7
:105930007105F9F0EC89FD8981E090E008A002C0D2
:10594000880F991F0A94E2F7808360E079E08DE385
:1059500090E0A70196010E949B2D21503109410939
:1059600051095695479537952795211580E13807B8
:1059700098F0EC89FD89108260E874E88EE190E08F
:10598000A70196010E949B2D21503109410951091F
:105990005695479537952795E889F9893083EA899F
:1059A000FB89208319A2EE89FF89408181E090E084
:1059B0009C010C8C02C0220F331F0A94E2F7422B89
:1059C0004083EE89FF8940819C010D8C02C0220F2B
:1059D000331F0A94E2F7422B4083EE89FF8940810E
:1059E0009C010E8C02C0220F331F0A94E2F7422B57
:1059F0004083EE89FF8920810F8C02C0880F991F98
:105A00000A94E2F7809582238083DF91CF91FF9003
:105A1000EF90DF90CF9008958F929F92AF92BF92B8
:105A2000CF92DF92EF92FF920F931F9381E08F93BB
:105A300085E08F9387E08F9383E08F9384E08F934B
:105A4000E6EC8E2E912CF2ECAF2EB12CA1ECCA2EEE
:105A5000D12CB0ECEB2EF12C04EC10E025EC30E076
:105A600042E056E066E476E080EE95E00E94592C34
:105A70000F900F900F900F900F901F910F91FF902C
:105A8000EF90DF90CF90BF90AF909F908F90089550
:105A90000E94A9280E941322C5E1DCE20E94AF24E3
:105AA0002097E1F30E94152CF9CFA29FB001B39F7C
:105AB000C001A39F700D811D1124911DB29F700D17
:105AC000811D1124911D08950E94552DA59F900DB3
:105AD000B49F900DA49F800D911D11240895B7FFD0
:105AE0000C94642D0E94642D821B930B0895DB019E
:105AF0008F939F930E94642DBF91AF91A29F800DC1
:105B0000911DA39F900DB29F900D1124089597FBB6
:105B1000072E16F4009407D077FD09D00E94192EA5
:105B200007FC05D03EF4909581959F4F08957095A0
:105B300061957F4F0895A1E21A2EAA1BBB1BFD01A0
:105B40000DC0AA1FBB1FEE1FFF1FA217B307E4075C
:105B5000F50720F0A21BB30BE40BF50B661F771FB4
:105B6000881F991F1A9469F7609570958095909594
:105B70009B01AC01BD01CF010895052E97FB1EF4DA
:105B800000940E94D42D57FD07D00E949B2D07FC46
:105B900003D04EF40C94D42D50954095309521951A
:105BA0003F4F4F4F5F4F0895909580957095619549
:105BB0007F4F8F4F9F4F08952F923F924F925F924A
:105BC0006F927F928F929F92AF92BF92CF92DF920D
:105BD000EF92FF920F931F93CF93DF93CDB7DEB772
:105BE000CA1BDB0B0FB6F894DEBF0FBECDBF099406
:105BF0002A88398848885F846E847D848C849B845D
:105C0000AA84B984C884DF80EE80FD800C811B816A
:105C1000AA81B981CE0FD11D0FB6F894DEBF0FBE99
:105C2000CDBFED010895EE0FFF1F0590F491E02D1B
:105C30000994AA1BBB1B51E107C0AA1FBB1FA617D3
:105C4000B70710F0A61BB70B881F991F5A95A9F725
:105C500080959095BC01CD0108958F929F92AF924F
:105C6000BF92CF92DF92EF92FF92CF93DF93EC013E
:105C7000688179818A819B81611571058105910512
:105C800021F464E279ED8BE597E02DE133EF41E01B
:105C900050E00E94BD2D49015A019B01AC01A7EAC9
:105CA000B1E40E94642D6B017C01ACEEB4EFA50160
:105CB00094010E94722DC60ED71EE81EF91EF7FE33
:105CC00006C081E0C81AD108E10880E8F80AC88255
:105CD000D982EA82FB82C701B6019F77DF91CF911B
:105CE000FF90EF90DF90CF90BF90AF909F908F90FC
:105CF00008950E942D2E089586E091E00E942D2E99
:105D000008956093060170930701809308019093B2
:105D1000090108952F923F925F926F927F928F9226
:105D20009F92AF92BF92CF92DF92EF92FF920F932A
:105D30001F93CF93DF938B01EA016115710521F069
:105D4000DB018C9311969C93209739F09E01225091
:105D500031092332310508F0D8C07C016701BFEF5B
:105D6000CB1ADB0A5601F7016080862D90E00E9475
:105D7000BC2F892B11F07601F1CFFDE26F120AC022
:105D8000570182E0A80EB11CD70111966C907724C0
:105D900073940BC0BBE26B1207C05701E2E0AE0E7A
:105DA000B11CD70111966C90712CCE018F7E892B7E
:105DB00089F4B0E36B1237C0F50180818F7D88359F
:105DC000D1F46180F2E0AF0EB11C872D8260782E95
:105DD000C0E1D0E0CA30D10551F1C031D10521F088
:105DE000C830D10599F409C0CC24CA94DC2CEC2C21
:105DF000AFE0FA2E22C0209769F7C8E0D0E0CC24AB
:105E0000CA94DC2CEC2CFFE1FF2E17C06FEF7FEF64
:105E1000CB019E01442737FD4095542F0E949B2DB6
:105E200069017A010AC02097A9F6CAE0D0E0E9E941
:105E3000CE2EDC2CEC2CE9E1FE2EF50160E020E01A
:105E400030E0A9014E01AA2497FCA094BA2C1F01AE
:105E500070ED572E560CA9E0A51570F48FEB860D4A
:105E60008A3118F499EC592E06C08FE9860D8A31D3
:105E700048F589EA582E560C852D90E08C179D0721
:105E80000CF56F3FD9F0C216D306E406F50698F07C
:105E9000C501B4010E94772D9B01AC01852D90E0D6
:105EA000A0E0B0E0280F391F4A1F5B1F28173907F1
:105EB0004A075B0710F46FEF01C061E03196D10132
:105EC0006C90C5CF0115110551F0662311F0319783
:105ED00003C071FE04C03297D801ED93FC9370FEAD
:105EE00007C050954095309521953F4F4F4F5F4FDC
:105EF00067FF10C082E290E090938B0680938A0641
:105F00006FEF7FEF8FEF9FEF07C060E070E080E002
:105F100090E002C0B901CA01DF91CF911F910F91AA
:105F2000FF90EF90DF90CF90BF90AF909F908F90B9
:105F30007F906F905F903F902F900895FC0188278D
:105F40009927E89421912032E9F3293010F02E307E
:105F5000C8F32B3241F02D3239F4689404C00E940A
:105F6000F02F820F911D219120532A30C0F31EF48F
:105F7000909581959F4F0895911150C0803219F0EE
:105F800089508550D0F7089548EC53E00E94C92FFE
:105F90000895FA01A191B081009719F41097E1F0EA
:105FA000CD01DC01CD010D90002011F4C00113C022
:105FB000FB012191222319F02015D9F7F3CFFB0122
:105FC0002191201519F41E92119606C02223C1F7C3
:105FD0000D900020A1F7D001FA01A193B08308959C
:105FE0007AE0979F902D879F802D910D1124089521
:105FF000F999FECF92BD81BDF89A992780B5089591
:10600000262FF999FECF1FBA92BD81BD20BD0FB6D4
:10601000F894FA9AF99A0FBE01960895992788275D
:066020000895F894FFCF83
:1060260000008C06200001000000FF0002000200B4
:10603600020002000200020002000200020002004A
:106046000200020002000200020002802500000594
:10605600400AA1204EA50020244EA52C2330C012B4
:1060660000001A400AA1204EA5001B1E27522C2311
:10607600308025000005400AA1204EA50020244EB0
:10608600A52C2330004B000006400AD0009D490095
:106096007B289D492C233000E1000005400A45017C
:1060A600D7DC03B81E0EBF00232E48E801008A4045
:1060B6000A6001555502AD1E20000023C854582021
:1060C60074696D656F75742100596573004E6F00B4
:1060D6002C00386368004E2F41002C205B005D20A9
:1060E60028002900486F70206368616E6E656C2019
:1060F6000020402000456E746572696E67206164F9
:10610600617074697665206368616E6E656C207374
:10611600656C656374696F6E2C207069636B696E5C
:10612600673A007363616E6E6572206D6F64650019
:106136004E4F5420454E41424C45440053656E64D3
:10614600696E672073657474696E677320746F2057
:1061560052580A00526573657474696E67207365D8
:106166007474696E6773206F6E2052580A0041621C
:106176006F727465642065646974730A00696E766B
:10618600616C69642073656C656374696F6E000D7C
:106196000A496E76616C696420696E707574202D8B
:1061A60020646973636172646564210700536574D2
:1061B60074696E677320736176656420746F204519
:1061C6004550524F4D0A00526576657274656420DB
:1061D60073657474696E67732066726F6D204545CA
:1061E60050524F4D0A004C6F6164656420666163CE
:1061F600746F72792064656661756C74730A004BFE
:10620600657920616E64206368616E6E656C7320CB
:1062160072616E646F6D697A65640A004F70656EAF
:106226004C52536E67205458207374617274696EB1
:10623600672000206F6E20485720006D6F64756CD4
:1062460065206C6F636B65643F00342B3400380047
:10625600382B340031320031322B340031360050C5
:10626600504D0052535349005344410053434C0090
:10627600525844005458440041494E004C4245454A
:10628600500053504B54524D0053425553005355F2
:106296004D44004C4C494E440000070B0C101115A0
:1062A60000B6012A032E033003340337033C03B63A
:1062B600013F03430348034C035003540358035C54
:1062C60003620369036E0373038C028C028C028CD7
:1062D60002160A13223129000000009D2BA2294331
:0862E6002B702B552B922B00AD
:107E00000F92CDB7DEB7112484B714BE81FFF1D035
:107E100082E08093C00088E18093C10086E0809377
:107E2000C20080E18093C4008EE0CDD088249924E4
:107E3000CC24C394F5E0DF2EE1E1EE2E73E0F72EC3
:107E4000B6D0082F813479F4B2D08983C2D0898129
:107E5000823811F481E005C0813811F485E001C059
:107E600083E09ED09AC0823411F484E103C085344B
:107E700019F485E0B6D091C0853561F498D0082F0B
:107E800010E095D090E0982E8824802A912A880CC2
:107E9000991C82C0863521F484E0A3D080E0E1CF34
:107EA000843609F04CC083D082D0A82E80D0B82E62
:107EB00000E011E07CD0F80181938F01AE16D1F77C
:107EC00088D0FB2DF53489F4E0E0F1E00BC0F9999E
:107ED000FECF92BC81BC0894811C911C819180BD15
:107EE000FA9AF99AEA1598F358C08B2D863409F05E
:107EF00054C0F401F7BEE89507B600FCFDCFF401CD
:107F0000A0E0B1E02C9130E011968C91119790E0B7
:107F1000982F8827822B932B12960C01C7BEE895C9
:107F20001124329681E0A038B80761F7F401D7BE7A
:107F3000E89507B600FCFDCFE7BEE8952EC0843774
:107F4000F1F435D034D0182F32D0B82E42D0FB2DDA
:107F5000F63421F4F40105914F010CC0FB2DF534EA
:107F600049F4F999FECF92BC81BC0894811C911C04
:107F7000F89A00B5802F14D0115049F70EC08537FC
:107F800039F427D08EE10CD085E90AD08FE069CF93
:107F9000813511F488E017D01CD080E101D050CF9A
:107FA0009091C00095FFFCCF8093C600089580910A
:107FB000C00087FFFCCF8091C00084FD01C0A89560
:107FC0008091C6000895E0E6F0E098E19083808318
:107FD0000895EDDF803219F088E0F5DFFFCF84E10E
:107FE000DFCF1F93182FE3DF1150E9F7F2DF1F9166
:0E7FF0000895282E80E0E7DFEE27FF27099492
:027FFE0001057B
:0400000300007E007B
:00000001FF
